:1000000012C018951895189564C2189518951895EA
:100010001895B8C0189518951895189518951895AD
:100020001895189518958FE58DBFC8E3E0E24E2E20
:1000300084E08EBFD4E0F4E05F2EA89584B7082E4C
:10004000877F84BF88E1992781BD91BDEEEFF3E002
:10005000A0E6B0E088278D933197E9F7662483E026
:1000600083BF79B7716079BF83E083BF85E886B9C4
:1000700080E487B9379A88E082BD85E085BD79B78D
:10008000706479BFAFE6B0E0E8E0F6E0FED1E9D118
:100090008FEF81BB7FE077BB70E074BBA89AA99A11
:1000A00080E080937D0080E080937E0089E78093EC
:1000B000800084E28093810080E38093820089E164
:1000C0008093830082E18093840082E080938500A6
:1000D00088E78093860080E08093870080E18093AA
:1000E000880080E4809389008CE180938A0086E414
:1000F00080938B0081E080938C0080E080938D0062
:100100007894999901C006D0989901C01FD0F9CF71
:10011000F894FFCF80E080937D0080E080937E00A4
:10012000A1E6B0E08C918F5F8C93009161000B335E
:1001300010F009F001C003C080E0809361008CE200
:1001400091E080D1999901C0E5CF089580E0809336
:100150007D0080E080937E00A2E6B0E08C918F5F0E
:100160008C9300916200073110F009F001C003C0C8
:1001700080E0809362008CE291E064D1989901C0A4
:10018000E5CF08950F921F922F923F924F925F9268
:100190007F92AF92BF920F931F932F933F934F93F2
:1001A0005F936F937F938F939F93AF93BF93CF93FF
:1001B000DF93EF93FF938FB78F9300917E00003012
:1001C00009F02EC000918C00013009F008C00091A8
:1001D00061004AE009D2AFE7B0E08C9320C0023062
:1001E00009F008C0009161004AE0FED1AFE7B0E03D
:1001F0000C9315C0043009F008C0009162004AE079
:10020000F3D1AFE7B0E08C930AC0083009F007C023
:10021000009162004AE0E8D1AFE7B0E00C9325C05E
:1002200000918C00013009F004C08CE080937F00C5
:100230001CC0023009F004C08BE080937F0015C021
:10024000043009F008C000917C004AE0CDD1AFE74E
:10025000B0E08C930AC0083009F007C000917C0020
:100260004AE0C2D1AFE7B0E00C9300917F000030CC
:1002700009F003C08AE080937F00AFE7B0E0AD9063
:10028000BB24AFE7B0E0AA0DBB1D8C9182BB00EF91
:1002900040918C00042B08BB00918C00043009F0C5
:1002A00010C000917E00003009F009C000918D005F
:1002B000003009F002C0979A01C0979801C0979842
:1002C00001C0979800918C00083081E009F080E02F
:1002D0008F93009162000A3081E008F080E09F91E6
:1002E0008923882309F406C000917E00003009F0BC
:1002F00001C0C39800918C00083008F005C091E05F
:10030000ACE8B0E0D0D003C081E080938C008F9146
:100310008FBFFF91EF91DF91CF91BF91AF919F91EF
:100320008F917F916F915F914F913F912F911F918D
:100330000F91BF90AF907F905F904F903F902F9024
:100340001F900F901895ADE7B0E08C918F5F8C9364
:1003500000917D00053010F009F001C009C080E077
:1003600080937D00AEE7B0E08C9191E089278C937B
:10037000ADE8B0E08C9191E089278C9300917E00EC
:10038000003009F018C007B1007F026007B982D0C1
:10039000A8E7B0E08D939C93A8E7B0E00D911C9185
:1003A00042E050E02CD0AAE7B0E04D935C938091FE
:1003B0007A0080937C00089500FC10D0089503D04B
:1003C0001ED001F8F9CF0024E89457FF02C009D0ED
:1003D000689400F80BD010F80124089502D009D0D9
:1003E0000895509540954F5F5F4F0895E89417FF2B
:1003F0000895009510950F5F1F4F68940895352F4D
:10040000242FE894452B11F468940895512F402F20
:100410000027112780E1440F551F001F111F021BE9
:10042000130B416018F4020F131F4E7F8A9599F742
:1004300008953197F1F70895689462F80895E89463
:1004400062F80895EF93FF93EE27E82BE92B31F044
:10045000E8EEF3E03197F1F70197D1F7FF91EF91D3
:100460000895EFE6F0E0A0E6B0E002C0ADE0BB2703
:100470008681978124D00D938381948120D00D9320
:10048000808191811CD00D93089515D00D9200208C
:10049000E1F70895369A3699FECF369A3699FECF0F
:1004A00084B195B10895903029F08C91880F9A9578
:1004B000E9F78C930895C8953196002008958053EC
:1004C00090530027813018F0065F8A95FBCF090F03
:1004D0000895AF93BF930F939F938F938FB78F938D
:1004E000A0E6B0E08C9183958D938C3309F03DC0EC
:1004F00088278E9311968C9183958D938C3309F078
:1005000034C088278E9311968C9183958D93883172
:1005100061F588278E9311968C9183958D939C918C
:100520000EE1943089F0963079F0993069F09B3083
:1005300059F00CE1923039F411969C911197937017
:1005400019F4039501C00FE1801778F071F081E094
:100550008E9311968C9183958D938D3031F481E03B
:100560008E9311968C9183958C938F918FBF8F91E1
:100570009F910F91BF91AF910F921F922F923F9237
:100580004F925F927F92AF92BF920F931F932F93E0
:100590003F934F935F936F937F938F939F93AF930B
:1005A000BF93CF93DF93EF93FF938FB78F93CBDE00
:1005B0008F918FBFFF91EF91DF91CF91BF91AF915D
:1005C0009F918F917F916F915F914F913F912F916B
:1005D0001F910F91BF90AF907F905F904F903F9091
:1005E0002F901F900F901895FF93881BF9E0001F24
:1005F000FA9511F4FF910895881F841B18F4840F55
:0E0600008894F5CF0894F3CF31323A333000AE
:00000001FF
